:020000040000FA
:060000000219FD0200C818
:03000B0002008D63
:03002B000200923E
:03005B000202C6D8
:030073000200B5D3
:100080000406080C10182030406080A0C0C28D0506
:100090004032C0D0C0E0C2CF0541E5646009E563ED
:1000A000600575630001B0756301E52360021523E7
:1000B000D0E0D0D032C2AF53E67F7592FA7593FF8D
:1000C000C22053917FD2AF32C0D0C0E0C0F0D2D3B3
:1000D0005388EFA88AA98CAA40308D010A758A003E
:1000E000758C00754000438810E564700AC3E833DE
:1000F000F8E933F9EA33FA30331FE8C4540FFAE968
:10010000C454F04AFAC3132AFAC3E833F8E933F9BE
:10011000E82AFAE93406FB216C30320FC3E833E9F0
:1001200033FAE82AFAE93400FB216C303115E8751E
:10013000F056A4AAF0E975F056A42AFAC5F03400E6
:10014000FB216CC3EA13FAE913F9E813F8E875F038
:1001500056A4AAF0E975F056A42AFAC5F03400C3F3
:1001600013FBEA13FAC3EB13FBEA13FAC3EB941283
:100170005006C3EB9406501A0522E52270021522A0
:10018000C3E522940A500241BC7552007A007B00FC
:10019000418DE522600215223035067C007D082164
:1001A000ACAC31AD32303A04AC33AD34C3EA9CFA76
:1001B000EB9DFB9208AE5EAF5F303A4250072034B1
:1001C00009D23421CA303402C234303404AE60AFB4
:1001D00061203902B234C3EA33FAEB33FBA2085090
:1001E0000AEAF42401FAEBF43400FBC3EA9450FA6F
:1001F000EB9400FB501478007A007B00410AA208BF
:10020000500878007A007B004169E5255403601BA3
:10021000202A18E55B33F9EB7007C3E99A4002E93D
:10022000FAE53CC4332AFAEB3400FBEA8EF0A4F979
:10023000AAF0EB8EF0A42AFAC5F03400FBC3EB134E
:10024000FDEA13F8C3ED13FDE813F80FEF14600493
:10025000C3E833F8C3E933EA33FAEB33FBDFEDEB02
:1002600030E30678FF7AFF7B078852D230C3E894E8
:10027000404002D221C3E559FC955A4003AC5AC311
:10028000EC95525008EC75F008A4FAABF0EAF4F8DB
:10029000EBF45407F9C3E89414FAE99400FB500412
:1002A0007A007B00885489558A568B5775230AD06B
:1002B000F0D0E0D0D053F7DF43F7403275230AD0B7
:1002C000F0D0E0D0D032C0D0C0E0D2D3A8F9E55809
:1002D00030E107E5FA30E2076114E5FA30E235C3B0
:1002E000E55513F8E55413F5FB88FCC3E55713F8FF
:1002F000E55613F5E988EA85555853F7BFC3E5522B
:10030000940140057553006114E5532401F55350E1
:10031000037553FF53F7DFD0E0D0D032790180145A
:1003200079038010790A800C791E80087964800432
:1003300079C880007817E4D5E0FDD8FAD9F6227A9A
:10034000147B7880127A107B8C800C7A0D7BB480C1
:10035000067A0B7BC880007902E4C291D5E0FDD219
:1003600090D5E0FDC290D5E0FDD291D5E0FDE92029
:10037000E002D28630E002D292E562D5E0FDE920CB
:10038000E002C28630E002C2927496D5E0FDD9C97F
:10039000EAF8D5E0FDD8FBDBBEC2912278FFC2218E
:1003A00020283D202912D221C3E548940A4009C3E0
:1003B000E55294405002C22179A1E76023E54860EC
:1003C0001F74FF8548F084853FF030290375F005E0
:1003D000A4F8C5F0600278FFC3E8955B5002A85B03
:1003E000885A22C3E54794A0E5489400E55A500393
:1003F0001461F4046002F55A2275E89022055CC38A
:10040000E55C94084055E5E820ECF2A8BDA9BE756E
:100410005C00E9FA79A0E76041EA7006E55D6018E2
:10042000800CC3E8955D600EE55D5005600A1480A0
:10043000070460FA8002E55DF55DC394F6401B7524
:1004400059C0C394064013755980C39406400B7578
:100450005940C39406400375590022E559241050B1
:100460000274FFF55922743279A687F0A4C5F0A270
:10047000F733F8C3E895594002A859885B227547BD
:10048000007548F022C2AF75C800A8CCA9CDAA411A
:1004900030CF010A75C804D2AFC3EA13FAE913F9E1
:1004A000E813F8AB42AC4388428943C3E89BF8E9C0
:1004B0009C20280A547FF9302C02A19F81FCAD4476
:1004C0008A44F9EA9D547FFA600478FF79FFAE45CB
:1004D000AF468B458C46A842A943C3E89EF8E99FE6
:1004E000F9C3E54813FBE54713FAE82AF547E93B6A
:1004F000F54850067547FF7548FFA146AA47AB4827
:10050000AC47AD487E047F02C3EB9404400A1E1F33
:10051000C3EB940840021E1FC3ED13FDEC13FCDE79
:10052000F7C3EA9CFAEB9DFBEF6009C3E913F9E816
:1005300013F8DFF7EA28FAEB39FB8A478B485006B5
:100540007BFF8B478B48C3EB94025002D22C3028A0
:10055000047F03A1717892E6FFC3E53D94824011C8
:100560000FC3E53D94A040010FC3EF940640027F06
:10057000057E02E548C4540FF9E548C454F0F8E597
:1005800047C4540F28F8C3E89EFAE99400FB4009D9
:10059000C3EA9401EB940050047A01E4FBA1EBAAB6
:1005A00047AB48EBC4FEEAC4540F4EFCC3EA9CFAC6
:1005B000EB9400FBC3E813C313F8EA28FAEB34000A
:1005C000FB8A478B48C3EB94024002C22C7802EBB3
:1005D000C4FE7B00EAC4540F4EFAC3EA98FA400501
:1005E000C3940150027A017892E6FF30200280FB2A
:1005F000854E92854F93D22043E680C3E49AF8E477
:100600009BF9C3E833F8E933F9302C02C17DE8FAED
:10061000E9FBD3E913FDE813FC884E894FC3EF943F
:10062000036037EF20E00CE82CF8E93DF9ECFAED37
:10063000FB8013E828F8E939F9C3E82401F8E93424
:1006400000F97AFF7BFFC3EF9403400E8A508B5171
:10065000884A894B8C4C8D4DC1B1885089518A4A4A
:100660008B4B8C4C8D4D3028127550F07551FF75A9
:100670004CF0754DFF754EF0754FFFC1B1E8FAD3E0
:10068000E813FC884EC3EF94036020EF20E007E8F6
:100690002CF8ECFAC19DE8282401F87AFFC3EF9406
:1006A0000340088A50884A8C4CC1B188508A4A8CD1
:1006B0004C302002C1B1753A02D22043E680E525D4
:1006C0005403602DA847A948C3E913F9E813F8308B
:1006D0002804E92440F9C2AF53E67F759100C3E4D2
:1006E00098F594E499F595759104D22043E680D26B
:1006F000AF22D222754900752000302B03752040AF
:10070000800ED222754900752040302B03752000E1
:1007100078017901202C20E52554036002C222795A
:1007200014E548C313700104F8C39414400278140C
:10073000302804781B791BC3E833F8C3E933F92068
:100740002010E549600C302803D53A04D224E1C7D3
:10075000D1B90549E59B5440B52002E1B1302809E3
:1007600008C3E899400118E13F20220A08C3E8992C
:100770004002E110E13FC222C2AF53E67F75910013
:10078000302C127594007595FC759104D22043E6C7
:1007900080D2AFE110AE47AF48C3EE33FEEF33FF78
:1007A00050047EFF7FFFC3E49EF594E49FF595E13E
:1007B00089C3E53994015002E110302202E110D8DA
:1007C00002E1C5E13FC224C2AF53E67F75910085C7
:1007D0005094855195759104854A92854B93D2200A
:1007E00043E680D2AFE5255403600720290205398E
:1007F000801030240D202B0A20220715811581023C
:100800000F1C2278003021053022027801E53D7569
:10081000F007A4F9E5F028F5F0E9A2F013A2F1132E
:10082000A2F213F53DC394785003753D78C3E53DBE
:10083000953E400ED223C286C290C29275D4FF75F7
:10084000D50F30200280FB854C92854D93D22043FA
:10085000E68022203813C2AFC291D28775D4FF75CB
:10086000D503D2AF759F42214BC2AFC291D29375CF
:10087000D43F75D50FD2AF759F42214B203814C29B
:10088000AFC29275D4FF75D50CD287D2AF759F5287
:1008900002094BC2AFC28675D4FF75D50CD293D274
:1008A000AF759F3202094B203813C2AFC287D29373
:1008B00075D4FF75D50CD2AF759F32214BC2AFC234
:1008C00093D28775D4FF75D50CD2AF759F52807BBC
:1008D000203814C2AFC29075D43F75D50FD293D2D1
:1008E000AF759F4202094BC2AFC29075D4FF75D558
:1008F00003D287D2AF759F4202094B203813C2AF93
:10090000C293D29175D43F75D50FD2AF759F5280E7
:100910003AC2AFC287D29175D4FF75D503D2AF75F5
:100920009F328027203813C2AFC28675D4FF75D599
:1009300003D291D2AF759F328011C2AFC29275D4EB
:100940003F75D50FD291D2AF759F52C22322C28676
:10095000C290C292C287C291C29375D4FF75D50F5F
:1009600022788076FF0876FF0876FF0876FF087603
:10097000FF0876FF0876090876FF087601788C76FE
:10098000010876FF0876FF0876FF0876FF0876FFF5
:100990000876030876FF0876FF0876FF08762508B4
:1009A00076D00876280876500876040876FF087610
:1009B000020876FF08767A0876FF08760108760145
:1009C0000876FF0876FF08760008760022FA75F0B0
:1009D0000CA4ABF0EAC333F8740133F9E8C333F87D
:1009E000E933F9E8C32BF8E93400F9E8C333F8E94F
:1009F00033F9227888E6C39403D23A5002C23AC24D
:100A000038E630E102D238A23892397886E614907E
:100A100000809378A6F67886E6F53FC394025003EB
:100A2000753F02789CE6753EFFB40203753EA0B4A4
:100A30000303753E827896E631CD88318932789EFF
:100A4000E631CD883389347897E631CD88358936DB
:100A5000314E223035117A007B007CFF7D007E0014
:100A600051BA8B5F8A5E22303A227896E6FA7B0092
:100A7000789EE6FC7D00C3EA33FAEB33FBC3EC332C
:100A8000FCED33FD7E0A51BA8B618A607896303A6C
:100A900002789EE6FA7B007897E6FC7D007E0030C7
:100AA0003A10C3EA33FAEB33FBC3EC33FCED33FD0E
:100AB0007E0A51BA8B5F8A5E2222C3EC9EFCED94C3
:100AC00000FDC3EC9AFCED9BFDC3EC9423ED940078
:100AD00050047C237D00C3EC94FFED940140047C22
:100AE000FF7D017BFF0B7A000AEA7009C3EC33FC3F
:100AF000ED33FD41E5EC8AF0A4AEF0ED8AF0A42ED2
:100B0000947C40E4EAF460DD22D23551531203288C
:100B10007A007B007C10120320E5522AFA74003B15
:100B2000FBDCF37C04C3EB13FBEA13FADCF7FFEB0B
:100B300060027FFFC23551532278A5E6F954037055
:100B400000E9540C7000E954307000E954C07000A2
:100B500022E5EF20E6037520000520903FFFE52009
:100B6000146006901DFF1460009304600375EF127B
:100B70007597DE7597AD7581C043FF8012031C75B4
:100B8000EF0275A900314E75803F75F1C375A4C0A1
:100B900075803F75D4FF75900075F20F75A50F75C0
:100BA000900075D50F75A60175E34075E202314ED0
:100BB000E4F8F6D8FD3161F15D7898866275300110
:100BC000C2AF12033012033F12032812034512036F
:100BD0002812034B1203287139C2AF78FA79FA3020
:100BE0008007D9FBD8F7021C0031F351537898865F
:100BF00062314E75A91375A71075C10075A70075F0
:100C0000640075E400758811758E0475890975C8CE
:100C10000475910475D84075D90875F782759E03DF
:100C200075960275DA4275DB4275A82375E69075F4
:100C3000F310759B80759D0075D12C75BCC075BB7C
:100C40001075E88075B20112031CD2AF753C00C26A
:100C500030120330C23175220012032CC3E52294F6
:100C60000A4024D231C23275220012032CC3E5227D
:100C7000940A4013D232C23375220012032CC3E50A
:100C800022940A4002D233120320203003020BD9EF
:100C9000C2AF12033F12033F12033FD2AF12033021
:100CA000303A02A133120320788CE6C3940150023B
:100CB000A133E530C394015002A1337F02D23551F4
:100CC0005312032CC2AFC2355153AE52C3E55294F6
:100CD0007FD2AF405E12031CC2AF120351D2AFDF0E
:100CE000DC7109C3EF7897F6120330F197121040C8
:100CF0007F0AD235515312032CC2AFC2355153AEC5
:100D000052C3E552947FD2AF50E612031CC2AF1219
:100D1000033F12032412033FD2AFDFD67109EF2441
:100D2000037896F6120330F19712106F12032C51CC
:100D30005361D912032C7801303A027805C3E55289
:100D400098400281A0C2AF12035112035112035105
:100D5000D2AF120330753000E4F537F5380537E5CA
:100D600037F4703E0538789AE678191460127832B4
:100D700014600D787D14600878FA146003753800EB
:100D8000C3E53898401C314E12031C1538753700E6
:100D900078998662C2AF120351D2AF7898866212F8
:100DA000032C120324E523700261D97801C3E552B4
:100DB0009840AA12032CE5237003020BD9C2AF316D
:100DC0004EE4D2AFE4F55CF524F525F53D755C08FD
:100DD00012031C1203F9E5E820ECFBA8BDA9BEE94B
:100DE0007001F8885D1203FD755C08C2AF7559FF8C
:100DF000120466855B59855B5AD2AF75A71075C121
:100E00003075A70075A903756401303A07C2383000
:100E10003402D238D22875390011FB312412047EF5
:100E200012048512047E12048512047E1207021138
:100E30000311531204851206F2202C0312039C3076
:100E40002C031203E31103117C1204851207021113
:100E50000311A71204851206F2110311D0120485A2
:100E6000120702110311FB1204851203F91206F294
:100E7000110331241203FD120485302827855B59A4
:100E800079187A0CC3E53999400EC228D2298A3BD9
:100E9000855B59855B5A800CC3E55294014003027F
:100EA0000E2CE12430291C202B19E53B147006C2BE
:100EB00029D22AC12CF53BC3E55294014003020E0E
:100EC0002C8061753C0078FA79A4E760027803C34E
:100ED000E55398504FE523604B303A1720380520F2
:100EE0003407800F303402800A202B07D22B855B19
:100EF00059C15678F0302B05855B597820C3E548F9
:100F0000985003020E2C302B1BC22BC238303402F7
:100F1000D238D229753B12855B59C12C053CE5526C
:100F20006002E127753C00C2AF314E752400752583
:100F30000075A91375A71075C10075A70075640029
:100F4000D2AF12032C314E78A4E66006D287D2913C
:100F5000D293C3E53C9404400261D9A158901A0D84
:100F60007820F1D3E520B4550AA3F1D3E520B4AA43
:100F70000280063161F197801D901A0378807B0A08
:100F8000F1D3A308DBFA901A0F788C7B1AF1D3A364
:100F900008DBFA901A2922C2AF121014F1EC901A51
:100FA000007410F1D8A37401F1D8A37420F1D89083
:100FB0001A0378807B0AF1D7A308DBFA901A0F781E
:100FC0008C7B1AF1D7A308DBFA12102812100390B9
:100FD0001A2922E493F622E6438F01538FFD75EF21
:100FE0000275B7A575B7F1F0538FFE22438F024308
:100FF0008F0175EF0275B7A575B7F1901A0DF05313
:101000008FFC22901A0D7455120FD8901A0E74AAE4
:10101000120FD8227A3079D07820901A40120FD34C
:10102000E520F709A3DAF6227A3079D0901A40E762
:10103000120FD809A3DAF8227C05120330DCFB2258
:10104000C2AF12033F12034512034B1203511203A6
:101050002412033F12034512034B120351120324BF
:1010600012033F12034512034B120351D2AF22C2A7
:10107000AF12035112034B12034512033F12032414
:1010800012035112034B12034512033F12032412A1
:0E109000035112034B12034512033FD2AF224D
:1019FD00020B51100120FFFFFFFFFFFF09FF01FF49
:101A0D0055AA01FFFFFFFFFF03FFFFFF25D0285061
:0D1A1D0004FF02FF7AFF0101FFFF0000FF40
:101A400023435F485F3130232020202020202020A6
:101A500023424C48454C492445464D3842323123B7
:101A60002020202020202020202020202020202076
:101C0000C2AFC2D37597DE7597AD7581C075A90057
:101C100043FF80752438752503B1C875EF0243F181
:101C20000153A4FED28075D4FF75E3407DFA78039A
:101C300079E67C10752200752300901DD57B067512
:101C400024987525013080028145208008D8FBD971
:101C5000F9DCF781B7308008D8FBD9F9DCF781B718
:101C6000B188E493A3C39A6004DDC381B7DBDBB121
:101C70007A6002812E7B08E493FAA3B15BDBF87AE9
:101C800030B15B752200752300B17AEAFCEBFDC32D
:101C9000ED94FE400EB17A8A278B28ED30E0048A5D
:101CA000828B83B17A7AC270D8C3ED94FE601350F0
:101CB000CEBD0023EC60097520007521FF020000F5
:101CC0008100A827A9280809D804D90281D4B17EA7
:101CD000EAF281C80D81A3C3ED94035047EDA2E061
:101CE00092007AC5C3E5829400E583941C5092204B
:101CF0000010438F02438F0175B7A575B7F1F0301F
:101D0000001DA827A9280809438F01538FFDD80477
:101D1000D902A11FE275B7A575B7F1F0A3A10E53C3
:101D20008FFC817F7AC1BD030CE493A3FAB13FDC41
:101D3000F8B137817F8181AA22AB23B15BEBFAEA4C
:101D40006222752608C3E52313F523E52213F52245
:101D500050066323A0632201D526EAB1C8B1C87535
:101D6000260AEAF4200102D280300102C280B1C802
:101D7000C3134002C201D526EB22B17EEAFB2080CC
:101D800002A17E308002A183752608AE24AF25C350
:101D9000EF13FFEE13FEB1CCB1C8C3EA13308002DB
:101DA0004480FA30E703632201C3E52313F523E5FA
:101DB0002213F52250066323A0632201D526D9E51C
:101DC0002265236523F52222AE24AF250E0FDEFE09
:101DD000DFFCD20122424C48656C6934373163E83C
:031DE000B2060147
:00000001FF
